:100000001FC00BC40AC409C408C407C406C405C47D
:1000100004C403C402C401C400C4FFC3FEC3FDC3BF
:10002000FCC3FBC3FAC3F9C3F8C3F7C3F6C3F5C3F4
:10003000F4C3F3C33F003F10803F103F1400082477
:1000400011241FBECFEFCDBFDFE3DEBFE4E3F0E05E
:1000500040E017C0B591A59135912591059107FD17
:100060000CC095918591EF01F92FE82F05900D9225
:10007000A217B307D9F7FE0104C01D92A217B30758
:10008000E1F7E034F40731F709D27DC3F894FFCFEC
:100090004F925F926F927F928F929F92AF92BF9298
:1000A000CF92DF92EF92FF92CF936B017C0123EE10
:1000B00038E34EE85FE3AFD34B015C0120E030E072
:1000C00040E85FE395D388230CF464C024E535E56C
:1000D00045E55FE3C701B6019ED32B013C0120E05B
:1000E0003FEF4FE757E488D318160CF03EC020E0EE
:1000F00030E04AE754E4C701B6018BD34B015C0101
:1001000024E535E540E554E486D36B017C0120E02D
:1001100030E040E85FE36CD388230CF120E03FEF50
:100120004FE757E4C701B60167D31816A4F420E0DF
:1001300030E040E251E4C501B4016DD3E0D1611576
:10014000710549F123E530E0C9010197F1F76150EC
:100150007109D1F720C0C701B601D1D102C061E059
:1001600070E0CB010197F1F716C020E030E04FE7D7
:1001700053E4C501B40140D318163CF4C301B201E5
:10018000BED1CB010197F1F709C0C501B401B7D1C8
:10019000C62F01C0C1E06C2F6A95F1F7CF91FF9097
:1001A000EF90DF90CF90BF90AF909F908F907F9017
:0801B0006F905F904F900895DD
:1001B8000BC0D7D240F0CED230F021F45F3F19F017
:1001C800EBC25111D6C21EC30CD298F39923C9F3BE
:1001D8005523B1F3951B550BBB27AA276217730745
:1001E800840738F09F5F5F4F220F331F441FAA1FF9
:1001F800A9F333D00E2E3AF0E0E830D091505040B9
:10020800E695001CCAF729D0FE2F27D0660F771F66
:10021800881FBB1F261737074807AB07B0E809F048
:10022800BB0B802DBF01FF2793585F4F2AF09E3FDD
:10023800510568F0B1C29DC25F3FECF3983EDCF314
:10024800869577956795B795F7959F5FC9F7880F56
:10025800911D9695879597F90895E1E0660F771FA8
:10026800881FBB1F621773078407BA0720F0621B39
:0E027800730B840BBA0BEE1F88F7E095089508
:100286000AC069D228F06ED218F0952309F085C20B
:10029600BAC211246FC2A6D1A0F3959FD1F3950FD0
:1002A60050E0551F629FF001729FBB27F00DB11DF4
:1002B600639FAA27F00DB11DAA1F649F6627B00D84
:1002C600A11D661F829F2227B00DA11D621F739F6D
:1002D600B00DA11D621F839FA00D611D221F749F7B
:1002E6003327A00D611D231F849F600D211D822FC2
:1002F600762F6A2F11249F5750408AF0E1F0882309
:100306004AF0EE0FFF1FBB1F661F771F881F915015
:100316005040A9F79E3F510570F03FC22BC25F3F88
:10032600ECF3983EDCF3869577956795B795F79548
:10033600E7959F5FC1F7FE2B880F911D96958795D0
:0403460097F9089586
:10034A00E89409C097FB3EF4909580957095619565
:10035A007F4F8F4F9F4F9923A9F0F92F96E9BB271B
:10036A009395F695879577956795B795F111F8CF97
:10037A00FAF4BB0F11F460FF1BC06F5F7F4F8F4F02
:10038A009F4F16C0882311F096E911C0772321F0F8
:10039A009EE8872F762F05C0662371F096E8862F90
:1003AA0070E060E02AF09A95660F771F881FDAF7E7
:0A03BA00880F9695879597F908952E
:1003C4000F931F93CF93DF93C82FD62F5FD1F1D113
:1003D4008C2F8FD1E091123FF091133F8C2F099510
:1003E4008C01ECD100511240083D114080F4EC2FF7
:1003F400F0E0E85FF04C8081811109C06D2F80E04E
:1004040094E09ED16D2F84E094E09AD10AC06D2FC0
:1004140084E094E07BD1EC2FF0E0E85FF04C81E0E5
:0C0424008083DF91CF911F910F9108950C
:100430000F931F93CF93DF93C82FD62F29D1BBD112
:100440008C2F59D1E091123FF091133F8C2F0995D9
:100450008C01B6D100511240083D114080F4EC2FC0
:10046000F0E0E050F14C8081811109C06D2F80E2F5
:1004700094E068D16D2F84E294E064D10AC06D2FBE
:1004800084E294E045D1EC2FF0E0E050F14C81E0C3
:0C0490008083DF91CF911F910F910895A0
:10049C0046D19AD1C6D0CCEAD7E806EB17E80F2E96
:1004AC00FAEDEF2EFAE1FF2EF02D98D1C70101974E
:1004BC00F1F78FD1899199910AD1C017D107A9F77A
:1004CC0088EA91E623E530E0F9013197F1F70197DD
:1004DC00D9F784D1CAEDDAE1CE010197F1F762E0E8
:1004EC0084E06ADF63E085E09DDF62E086E09ADF0E
:0204FC00F3CF3C
:1004FE007DD088F09F5790F0B92F9927B751A0F073
:10050E00D1F0660F771F881F991F1AF0BA95C9F799
:10051E0012C0B13081F029D1B1E0089526C1672F04
:10052E00782F8827B85F39F0B93FCCF38695779549
:10053E006795B395D9F73EF4909580957095619532
:08054E007F4F8F4F9F4F08956E
:100556000F931F93CF93DF931AD1E091123FF0913F
:10056600133F87E009958C0128D111D1E091123F04
:10057600F091133F87E00995EC011FD1C11582E088
:10058600D80730F081E0C017D10718F480E001C029
:0C05960080E0DF91CF911F910F9108953C
:1005A200990F0008550FAA0BE0E8FEEF1616170682
:1005B200E807F907C0F012161306E407F50798F0EA
:1005C200621B730B840B950B39F40A2661F0232B03
:1005D200242B252B21F408950A2609F4A140A6957F
:0805E2008FEF811D811D0895BA
:1005EA0057FD9058440F551F59F05F3F71F04795DA
:1005FA00880F97FB991F61F09F3F79F087950895BF
:10060A00121613061406551FF2CF4695F1DF08C0DD
:10061A00161617061806991FF1CF869571056105FA
:04062A000894089593
:10062E0060E080E096E0E8D065E081E096E0E4D01E
:10063E0064E082E096E07FD062E082E096E07BD0DC
:10064E0060E483E096E0BAD064E083E096E073D095
:02065E000895FD
:1006600061E088E096E0CFD0E0E0F6E0838580FFAF
:10067000FDCFE0E0F6E081E083878089918996955F
:100680008795929582958F7089279F708927089505
:10069000CF93883078F4C82F682F80E094E038D06A
:1006A0006C2F84E094E034D08C2F90E064E0805F85
:0806B0009B4F48D0CF91089543
:1006B800092E0394000C11F4882352F0BB0F40F468
:1006C800BF2B11F460FF04C06F5F7F4F8F4F9F4FA8
:0206D800089583
:1006DA00BC0180E090E034DEE091103FF091113FE0
:0C06EA00099561E084E094E00ED00895D2
:1006F600CF93883040F4C82F86E096E07ED06C2FEA
:0A07060086E096E07DD0CF910895C3
:1007100021E030E002C0220F331F6A95E2F72095F6
:0A072000FC0130812323208308959B
:10072A0062E084E094E0EFDF63E084E294E0EBDFF0
:0A073A0062E084E294E0E7DF089536
:1007440021E030E002C0220F331F6A95E2F7FC017A
:080754003081232B208308955E
:0E075C0000240A9416161706180609060895BA
:0E076A0000240A9412161306140605060895BC
:0E077800E894BB2766277727CB0197F90895F1
:0E078600EC014AD048D0CE0148D0CE0147D079
:0C07940087E07CDF87E0ADDF0CD008952B
:0C07A00097F99F6780E870E060E0089522
:0A07AC00FA00F401EE02E803E20493
:0A07B60060E080E096E0C3DF0895E4
:0A07C00060E080E096E0A4DF0895F9
:0A07CA00FC012081622B608308957A
:0A07D40061E080E094E0B4DF0895D6
:0A07DE0061E084E094E0AFDF0895CD
:0807E800B6DE8823E9F3089551
:0807F000D8DE08F481E0089551
:0807F800D4DE08F48FEF089530
:06080000FC0110820895C6
:06080600FC01608308956F
:06080C009FEF80EC08954F
:04081200D2DC51CF14
:0408160037DD4FCFAC
:02081A00F2CB1F
:02081C0008953D
:02081E0008953B
:02082000089539
:0208220034DCC4
:0208240048008A
:0208260030039D
:00000001FF
